:020000040000FA
:020000001E28B8
:040002000034003492
:08000800A000030E8312A10009
:100010002408A2002508A3000515AB202708A4008A
:100020000000A40B102805112208A4002308A50035
:100030000B11210E8300A00E200E090083128501F2
:100040000730990083169F012830850020309500E5
:100050002030960005308100FF23900083128B171B
:100060008B168B110B1005120511AA011D30A7006C
:10007000051690202A08AB000310AB0DAB0DAB0D9D
:10008000AB0D02308A002B080022FF3903196728C4
:10009000A800AB0A02308A002B080022A900AB0A94
:1000A0002808FF3A031961282908A600A70A851A1B
:1000B0006728AB20A60B592827082806031D5428BB
:1000C0004128A020851A6728A90B61284128A02073
:1000D000A020A020851E6A28AA0A2A080F3A031920
:1000E000AA010230A600A703AB20A60B742827089C
:1000F0001D3A031D7128A020A020A020A020851E4D
:100100003A28051283288B138B150B1005080B1842
:1001100085286300000005080B108B118B17382809
:100120000730A4002F30A5000330A600A40B9928A7
:10013000A50B9B28A60B96289D289E289F28080083
:100140001E30A4004F30A500A40BA728A50BA4289F
:10015000A92800000800C730A4000130A500A40BA6
:0A016000B228A50BAF28B428080050
:10040000820760340834FF340534BF3401340034CB
:10041000003400340034003400340034003400343C
:10042000003480340534FF340A34BF3401340034DE
:10043000003400340034003400340034003400341C
:100440000034BF340234003400340034003400344B
:1004500000340034003400340034003400340034FC
:100460000034BF340134003400340034003400342C
:1004700000340034003400340034003400340034DC
:10048000003440340434FF34053490340234FF34F3
:100490000A34BF34013400340034003400340034F2
:1004A000003460340834FF340534BF340134003480
:1004B000003400340034003400340034003400349C
:1004C0000034BF34043400340034003400340034C9
:1004D000003400340034003400340034003400347C
:1004E0000034FF34143490340534FF340A34BF34FC
:1004F000013400340034003400340034003400345B
:10050000003490340534FF342034BF3401340034D7
:10051000003400340034003400340034003400343B
:100520000034BF340134003400340034003400346B
:10053000003400340034003400340034003400341B
:100540000034FF34203430340434FF342034BF34DA
:1005500001340034003400340034003400340034FA
:100560000034BF3404340034003400340034003428
:1005700000340034003400340034003400340034DB
:100580000034BF340234003400340034003400340A
:1005900000340034003400340034003400340034BB
:1005A0000034FF343034BF340434003400340034B9
:1005B000003400340034003400340034003400349B
:1005C0000034BF34023400340034003400340034CA
:1005D000003400340034003400340034003400347B
:1005E0000034FF34143490340534FF340A34BF34FB
:1005F000013400340034003400340034003400345A
:020600000034C4
:02400E0084012B
:00000001FF
